:020000040000FA
:0404000064EF03F0B2
:020404000000F6
:0404080069EF02F0A6
:08041800E8CF89F0D8CF8AF08B
:10042000E0CF8BF0EACF83F0E9CF84F0E2CF85F024
:10043000E1CF86F0DACF87F0D9CF88F09DAA02D03D
:100440009EBA3BEC02F09DA802D09EB861EC02F08F
:1004500087C0DAFF88C0D9FF85C0E2FF86C0E1FF10
:1004600083C0EAFF84C0E9FF8BC0E0FF89C0E8FFDA
:100470008AC0D8FF1000ABA403D082BE01D0FF0019
:10048000AECF09F0ABB2AB9800000000AB8807B468
:10049000120010C0E2FF11C0E1FF09C0E6FF050E27
:1004A000E218D8B413EE00F00E50E26204D00F5000
:1004B000E16201D00784E2CF10F0E1CF11F007969E
:1004C000120007B204D08BEC02F0AD6E12009D98C2
:1004D0001200F2943D0ED66E2D2E1100640E2D6E7C
:1004E0002A662A062B662B06110007B012009D987B
:1004F0000B6E020EE26E0DC0E1FF0BC0E7FFFF0EB8
:100500000D18000ED8A40D280D6E0C5CD8B4078011
:1005100007929D881200020EE26E0CC0E1FFFF0EF2
:100520000C18000ED8A40C280C6E07900D18D8B427
:100530000782E750120007B612009D9A07940EC07A
:10054000E2FF0FC0E1FFE6CF0AF0050EE218D8B4D3
:1005500013EE00F01050E26204D01150E16201D0BD
:100560000786E2CF0EF0E1CF0FF00A509D8A12000D
:1005700007B603D09BEC02F0120000EC2DF007B69A
:1005800000EC2DF007B600EC2DF007B600EC2DF0D6
:1005900007B600EC2DF007B603D09BEC02F012007A
:1005A000060005D007B6FED79BEC02F01200E1EC86
:1005B0002AF0E3EC2AF0196A120007B603D09BEC8C
:1005C00002F0120000EC2DF007B600EC2DF007B69B
:1005D00000EC2DF007B603D09BEC02F012000600F1
:1005E000060006000DD00A0E2B6E2B6604D0060006
:1005F0000600060005D007B6F8D79BEC02F0120003
:100600002CEC03F061EF07F007B603D09BEC02F08F
:10061000120000EC2DF007B600EC2DF007B600EC50
:100620002DF007B603D09BEC02F012000600060086
:1006300006000DD00A0E2B6E2B6604D006000600B5
:10064000060005D007B6F8D79BEC02F012002CECA0
:1006500003F0196A6DEF08F0D40EB8EC2CF06E0EB2
:10066000F66E350EF76E000EF86E140E036E09006E
:10067000F550A0EC2CF0032EFAD71200000E0C6EF1
:100680000D6E07900782120013EE00F0E2CF0EF01D
:10069000E1CF0FF0E2CF10F0E1CF11F00794078621
:1006A0001200A69EA69CA680A8501200A69EA69CFC
:1006B000A684F29E550EA76EAA0EA76EA682F28E93
:1006C000A6B2FED7A6941200196A076A086A156ACC
:1006D000166A176A2E6A2F6A306AF16A566A000132
:1006E000806B826B940E0001816F640E2D6E15EC91
:1006F00004F01EEC04F00101576B05EE00F0EACFA8
:10070000E8F0E9CFE9F0EACFEAF0E9CFEBF00F0E3D
:10071000C16E806A896A926A898A816A8A6AFF0ED2
:10072000936E826A8B6A900E946E3EEC03F044ECFA
:1007300003F0AB6AAC6AB06A080EB86E200EAF6EFA
:10074000AE50AD6A9D8AAB8EAB88AC8A9F6AC70EED
:10075000D56E3D0ED66EF184800ED06EE00EF26E38
:10076000800EC76E310EC66E8FEC2AF0899A0F0E7E
:10077000F8EC03F002EC04F0898AE8AE11D0899A13
:100780000E0EF8EC03F002EC04F0898AE8BE03D008
:100790006AEC27F005D0440E136E0F0E59EC29F0C9
:1007A0000A0E2A6E000EAA6E000EA96E51EC03F01E
:1007B000A8CF1FF01EEC2DF0B6EC2AF02B6A2A50C1
:1007C000D8B463EC22F0E7EC28F02CAE86EC06F00F
:1007D0002CAC6AEC08F02CA492EC1EF02CA05FEC80
:1007E00005F02CA85FEC05F007A6FAEC1AF0E7D7A5
:1007F000576EEEEC2CF05750C96EC7A0FED7C9500B
:100800009E961200EEEC2CF0330EC96EC7A0FED7F8
:10081000C9509E961200899A0F0EF8EC03F002EC74
:1008200004F0898AE8B4F7D71200140E046E01EEC2
:1008300058F0200EEE6E042EFDD71200046801EE73
:1008400000F0200EEE6E042EFDD71200FE0E75ECA9
:1008500002F0FE0E75EC02F07F0E75EC02F0010E58
:1008600075EC02F01D0E75EC02F01200FE0E75EC38
:1008700002F0FE0E75EC02F07F0E75EC02F0010E38
:1008800075EC02F0200E75EC02F01200FD0E75EC16
:1008900002F0120026EC04F0070E75EC02F046ECB4
:1008A00004F0120026EC04F0080E75EC02F046ECA1
:1008B00004F0120026EC04F0090E75EC02F046EC90
:1008C00004F0120026EC04F00A0E75EC02F046EC7F
:1008D00004F0120036EC04F0020E75EC02F046EC67
:1008E00004F0120036EC04F0030E75EC02F046EC56
:1008F00004F0120036EC04F00F0E75EC02F046EC3A
:1009000004F0120036EC04F00C0E75EC02F046EC2C
:1009100004F0120036EC04F00A0E75EC02F046EC1E
:1009200004F0120036EC04F00B0E75EC02F046EC0D
:1009300004F0120036EC04F0070E75EC02F046EC01
:1009400004F0120036EC04F0060E75EC02F046ECF2
:1009500004F0120036EC04F0100E75EC02F046ECD8
:1009600004F012003DEC0DF0F3EC02F0D5EC1AF0BF
:10097000F3EC02F0336E94EC2BF0300EA0EC2CF084
:100980006D0EA0EC2CF0530EA0EC2CF0650EA0EC3C
:100990002CF0630EA0EC2CF061EF22F0C00EB8EC4E
:1009A0002CF04AEC0DF01AEC03F0020A02E0D7EF4B
:1009B00002F0140E036E1AEC03F0046E1AEC03F04E
:1009C000A0EC2CF004061CE0032EF8D7940EB8EC33
:1009D0002CF0140E036E1AEC03F0A0EC2CF00406BD
:1009E0000FE0032EF8D7D40EB8EC2CF0140E036EE3
:1009F0001AEC03F0A0EC2CF0040602E0032EF8D76A
:100A000061EF22F036EC04F0040E75EC02F046ECD7
:100A100004F0120036EC04F0090E75EC02F046EC1E
:100A200004F0120036EC04F0080E75EC02F046EC0F
:100A300004F012003DEC0DF0F3EC02F0D5EC1AF0EE
:100A4000F3EC02F0346E94EC2BF0300EA0EC2CF0B2
:100A5000530EA0EC2CF0650EA0EC2CF0630EA0EC75
:100A60002CF0200EA0EC2CF061EF22F03DEC0DF00C
:100A7000F3EC02F0D5EC1AF0F3EC02F03A6E5EEC17
:100A80002BF04EEC2BF061EF22F03DEC0DF0F3EC8F
:100A900002F0D5EC1AF0F3EC02F0366EF3EC02F053
:100AA000C00B376E060E036ED89036323732032EE7
:100AB000FCD7DCEC2BF051EC2BF061EF22F00001C5
:100AC00056B01AD0E851EA6317D0E951EB6314D05D
:100AD000D40EB8EC2CF0320EF66E350EF76E000E1A
:100AE000F86E140E036E0900F550A0EC2CF0032EE6
:100AF000FAD7020E2A6E12001EEC2DF0040EB8EC8E
:100B00002CF0E8C0EAFFE9C0E9FFED502CB807D0AF
:100B1000260E036EED50032EFDD73FEF06F0080EB4
:100B2000036EC70EB8EC2CF0ED50A0EC2CF0032EA9
:100B3000FBD7080E036ED10EB8EC2CF0ED50A0ECF4
:100B40002CF0032EFBD7080E036EA50EB8EC2CF08C
:100B5000ED50A0EC2CF0032EFBD7080E036E9B0E7D
:100B6000B8EC2CF0ED50A0EC2CF0032EFBD7910E3E
:100B7000B8EC2CF0EDCF12F012500F0B3009A0ECB6
:100B80002CF012380F0B3009A0EC2CF02F0EA0EC3B
:100B90002CF0EDCF12F012500F0B3009A0EC2CF01E
:100BA00012380F0B3009A0EC2CF02F0EA0EC2CF01B
:100BB000EDCF12F012500F0B3009A0EC2CF01238D0
:100BC0000F0B3009A0EC2CF0200EA0EC2CF0200E26
:100BD000A0EC2CF0EDCF12F012500F0B3009A0EC6E
:100BE0002CF012380F0B3009A0EC2CF03A0EA0ECD0
:100BF0002CF0EDCF12F012500F0B3009A0EC2CF0BE
:100C000012380F0B3009A0EC2CF03A0EA0EC2CF0AF
:100C1000EDCF12F012500F0B3009A0EC2CF012386F
:100C20000F0B3009A0EC2CF0060EB8EC2CF0E3EC26
:100C30002AF0EE500001EA51EA6214D0EB51E96269
:100C400011D0D40EB8EC2CF05A0EF66E350EF76EAD
:100C5000000EF86E140E036E0900F550A0EC2CF097
:100C6000032EFAD7040EB8EC2CF0ED50E7EC28F088
:100C70002CAA27D02CA803D02CA029D0F7D70E0E51
:100C8000EA6206D0F10EE96203D005EE25F047D7FF
:100C9000260E036EEE50032EFDD7E8C0DAFFE9C042
:100CA000D9FFDD50DA50EA6206D0D950E96203D0AC
:100CB00005EE25F034D7260E036EEE50032EFDD739
:100CC0002ED7060EB8EC2CF092EC1EF01200EAC003
:100CD000DAFFEBC0D9FFDD50040EEA6206D0FF0E4A
:100CE000E96203D056B081EC06F0DA50EA6217D719
:100CF000D950E96214D7E8C0EAFFE9C0E9FFED5036
:100D00000ED70F0EEA6E170EE96E1200800E036EFC
:100D100015EC2DF081BED2D015EC2DF081BECED0D9
:100D200015EC2DF081BECAD0032EF2D799EC06F057
:100D300012001EEC2DF0800EB8EC2CF00C0EB8EC6E
:100D40002CF00A0EF66E350EF76E000EF86E140ECD
:100D5000046E0900F550A0EC2CF0042EFAD73050A8
:100D600041E000D0140E036E000EF86E4F0EF76EC9
:100D7000C00EF66E0900F550A0EC2CF0032EFAD749
:100D80004CEC0BF081AEFED7E7EC28F02CA4DDEFA5
:100D900006F02CAAA5D02CB606D03006D8B0C9D7FC
:100DA000010E306EC6D72CB2EFD7302A020E3018A3
:100DB000D8A4BFD7306ABDD7E7D76CEC27F04CEC8E
:100DC00007F0E7EC28F02CAAB4D72CA6B2D72CA2B7
:100DD000B0D72CA8AED72CA0ACD72CB4F2D7E3EC6C
:100DE0002AF0EBD7C00EB8EC2CF01E0EF66E350EC6
:100DF000F76E000EF86E140E046E0900F550A0ECAC
:100E00002CF0042EFAD71FC058F0FDEC17F058B0A4
:100E100003D0FAEC2AF002D0EEEC2AF081AEFED735
:100E2000E7EC28F02CA413D02CAA5AD02CB606D06C
:100E30003006D8B07ED7010E306E7BD72CB2F0D7FB
:100E4000302A020E3018D8A474D7306A72D758EC02
:100E500008F0E7EC28F02CA858702CA058702CA4AF
:100E60000ED02CAA99EF06F0A00EB8EC2CF058B0DA
:100E700003D0FAEC2AF0EDD7EEEC2AF0EAD758C00E
:100E80001FF01FC0A8FF000EAA6E000EA96E56EC40
:100E900003F04CEC07F0DDD7D40EB8EC2CF0140EB8
:100EA000046EA60EF66E340EF76E000EF86E090094
:100EB000F550A0EC2CF0042EFAD712001EEC2DF009
:100EC00012D0E7EC28F02CAA0BD02CA494D02CA2A2
:100ED00080D02CA684D02CA88BD02CACFBD0F1D702
:100EE00092EC1EF01200E1EC2AF0E3EC2AF0800E06
:100EF000B8EC2CF00C0EB8EC2CF01E0EF66E300E8A
:100F0000F76E000EF86E140E046E0900F550A0EC9A
:100F10002CF0042EFAD7C00EB8EC2CF0000EFB6EAD
:100F20000F0EFA6E2E50E846E846036E3A0E032482
:100F3000D8B0FA2AD8B0FB2AF96EABEF0CF0C1EFAB
:100F40000CF003EF0DF0D7EF0CF057EF0DF0ADEF15
:100F50000DF004EF0EF01AEF0EF0EDEF0CF030EFA5
:100F60000EF046EF0EF05CEF0EF072EF0EF088EF31
:100F70000EF09EEF0EF00AEF0FF0A9EF0FF051EF19
:100F800010F0F9EF10F0A5EF11F04DEF12F0F5EFC2
:100F900012F09DEF13F0E7EF13F019EF14F04BEFA1
:100FA00014F07DEF14F0AFEF14F0E1EF14F013EF55
:100FB00015F045EF15F077EF15F0A9EF15F0DCEF20
:100FC00015F00EEF16F040EF16F072EF16F011EF7D
:100FD00017F02E2A260E2E602E6A73EF07F02E5081
:100FE00003E02E0673EF07F0250E2E6E73EF07F069
:100FF0002E6A73EF07F058EC08F0000EFB6E100E2F
:10100000FA6E2E50E846E846036E180E0326000ED0
:10101000FA22FB220350F96EE8EF22F03FEF23F0B3
:1010200071EF23F0E5EF23F089EF0DF0DFEF0DF026
:1010300007EF24F02BEF24F0A3EF23F04FEF24F081
:1010400073EF24F097EF24F0BCEF24F0E9EF24F0E5
:10105000D8EF0EF03CEF0FF0DAEF0FF082EF10F068
:101060002CEF11F0D6EF11F07EEF12F026EF13F017
:101070000EEF25F088EF25F0ADEF25F0D2EF25F04B
:10108000F7EF25F01CEF26F041EF26F066EF26F093
:101090008BEF26F0B0EF26F0D5EF26F0FBEF26F031
:1010A00020EF27F045EF27F0A4EF16F043EF17F0FD
:1010B000D40EB8EC2CF0140E046ECE0EF66E340E78
:1010C000F76E000EF86E0900F550A0EC2CF0042E1F
:1010D000FAD712001EEC2DF010D0E7EC28F02CAA65
:1010E00009D02CA252D02CA656D02CA85DD02CAE64
:1010F0000DD6F3D792EC1EF01200E1EC2AF0E3ECEF
:101100002AF0800EB8EC2CF00C0EB8EC2CF0320E5D
:10111000F66E300EF76E000EF86E140E046E0900B7
:10112000F550A0EC2CF0042EFAD7C00EB8EC2CF041
:10113000000EFB6E110EFA6E2F50E846E846036E65
:101140004E0E0324D8B0FA2AD8B0FB2AF96ED7EF96
:1011500008F00EEF09F05BEF0BF073EF0BF08BEF85
:101160000BF040EF0AF003EF0CF01BEF0CF0EBEF8D
:101170000BF0D3EF0BF0BBEF0BF0A3EF0BF03BEF5B
:101180000CF051EF0CF07EEF0CF02F2A0F0E2F60B9
:101190002F6A7DEF08F02F5003E02F067DEF08F057
:1011A0000E0E2F6E7DEF08F02F6A7DEF08F0140E03
:1011B000046E460EF66E300EF76E000EF86E0900E5
:1011C000F550A0EC2CF0042EFAD744EC03F0EFEC31
:1011D00008F0FDEC17F0F7EC08F06DEF08F026ECE6
:1011E00004F0030E75EC02F046EC04F0120034EC4F
:1011F0000BF0FF0AD8B412001AEC03F0030AD8A4CB
:101200001200080E036E1AEC03F0E86601D0200EFF
:10121000A0EC2CF0032EF7D7196A1200140E046EFE
:101220005A0EF66E300EF76E000EF86E0900F5508D
:10123000A0EC2CF0042EFAD744EC03F026EC09F0D5
:10124000FDEC17F02EEC09F06DEF08F026EC04F041
:10125000DC0E75EC02F046EC04F0120034EC0BF0FE
:10126000FF0AD8B412001AEC03F0DC0AD8A412006A
:10127000040E036E1AEC03F0E86601D0200EA0EC19
:101280002CF0032EF7D751EC2BF0196A120034EC36
:101290000BF0FF0AD8B412001AEC03F0070AD8A426
:1012A0001200080E036E1AEC03F0E86601D0200E5F
:1012B000A0EC2CF0032EF7D7196A120034EC0BF0D7
:1012C000FF0AD8B412001AEC03F0080AD8A4D7EF2A
:1012D00002F0080E036E1AEC03F0E86601D0200E4F
:1012E000A0EC2CF0032EF7D7196A120034EC0BF0A7
:1012F000FF0AD8B412001AEC03F0090AD8A41200AD
:10130000080E036E1AEC03F0E86601D0200EA0EC84
:101310002CF0032EF7D7196A120034EC0BF0FF0AF9
:10132000D8B412001AEC03F0010AD8A41200FDECA4
:1013300017F01AEC03F072EC2CF0200EA0EC2CF05D
:101340001AEC03F072EC2CF0200EA0EC2CF01AEC4E
:1013500003F072EC2CF0196A120034EC0BF0FF0A67
:10136000D8B412001AEC03F0010AD8A412001AEC47
:1013700003F01AEC03F01AEC03F0080E036E1AECFB
:1013800003F0E86601D0200EA0EC2CF0032EF7D776
:10139000196A120034EC0BF0FF0AD8B412001AECF0
:1013A00003F0010AD8A412000B0E036E1AEC03F02E
:1013B000032EFCD7080E036E1AEC03F0E86601D08A
:1013C000200EA0EC2CF0032EF7D7196A120034EC93
:1013D0000BF0FF0AD8B412001AEC03F0010AD8A4EB
:1013E0001200130E036E1AEC03F0032EFCD7080E46
:1013F000036E1AEC03F0E86601D0200EA0EC2CF08E
:10140000032EF7D7196A120034EC0BF0FF0AD8B498
:1014100012001AEC03F0010AD8A412001B0E036E8E
:101420001AEC03F0032EFCD7080E036E1AEC03F03F
:10143000E86601D0200EA0EC2CF0032EF7D7196A35
:10144000120034EC0BF0FF0AD8B412001AEC03F0CF
:10145000010AD8A41200230E036E1AEC03F0032E27
:10146000FCD7040E036E1AEC03F0E86601D0200EE0
:10147000A0EC2CF0032EF7D751EC2BF0196A1200D8
:10148000140E046EAA0EF66E300EF76E000EF86E95
:101490000900F550A0EC2CF0042EFAD744EC03F030
:1014A00062EC04F0FDEC17F058EC0AF06DEF08F078
:1014B00034EC0BF0FF0AD8B412001AEC03F00A0A5D
:1014C000D8A41200FDEC17F01AEC03F072EC2CF02B
:1014D000200EA0EC2CF01AEC03F072EC2CF0200E95
:1014E000A0EC2CF01AEC03F072EC2CF0196A12004C
:1014F0001CEC0BF0FF0AD8B41200D2EC02F00F0A79
:10150000D8A41200FDEC17F0D2EC02F03D6EE866B4
:101510009EEF17F0A3EF17F01CEC0BF0FF0AD8B406
:101520001200D2EC02F00C0AD8A41200FDEC17F065
:10153000D2EC02F03E6EE8669EEF17F0A3EF17F0D4
:101540001CEC0BF0FF0AD8B41200D2EC02F00A0A2D
:10155000D8A41200FDEC17F0D2EC02F03F6EE86662
:101560009EEF17F0A3EF17F01CEC0BF0FF0AD8B4B6
:101570001200D2EC02F00B0AD8A41200FDEC17F016
:10158000D2EC02F0406EE8669EEF17F0A3EF17F082
:101590001CEC0BF0FF0AD8B41200D2EC02F0070AE0
:1015A000D8A41200FDEC17F0D2EC02F0416EE86610
:1015B0009EEF17F0A3EF17F01CEC0BF0FF0AD8B466
:1015C0001200D2EC02F0060AD8A41200FDEC17F0CB
:1015D000D2EC02F0426EE866A8EF17F0C2EF17F007
:1015E0001CEC0BF0FF0AD8B41200D2EC02F0100A87
:1015F000D8A41200FDEC17F0D2EC02F0436EE866BE
:101600001AEF2BF00AEF2BF0B8EC02F0FE0AD2EC46
:1016100002F0FE0AD8A4FF0CD2EC02F0010AD8A412
:10162000FF0CD2EC02F07F0AD8A4FF0CD2EC02F03F
:101630001D0AD8A4FF0C000CDDEC02F0FE0AF3EC4E
:1016400002F0FE0AD8A4FF0CF3EC02F0010AD8A4C1
:10165000FF0CF3EC02F07F0AD8A4FF0CF3EC02F0CD
:10166000200AD8A4FF0C000C04EC03F0FE0A1AECCC
:1016700003F0FE0AD8A4FF0C1AEC03F0010AD8A468
:10168000FF0C1AEC03F07F0AD8A4FF0C1AEC03F04D
:10169000200AD8A4FF0C000CA4EC27F0120E036E55
:1016A00001EE3CF0940EB8EC2CF0EE50A0EC2CF0D7
:1016B000032EFBD71200140E046E6E0EF66E300E63
:1016C000F76E000EF86E0900F550A0EC2CF0042E19
:1016D000FAD744EC03F04AEC04F0FDEC17F047ECC9
:1016E00009F06DEF08F0140E046E820EF66E300EE7
:1016F000F76E000EF86E0900F550A0EC2CF0042EE9
:10170000FAD744EC03F052EC04F0FDEC17F05EEC79
:1017100009F06DEF08F0140E046E960EF66E300EA2
:10172000F76E000EF86E0900F550A0EC2CF0042EB8
:10173000FAD744EC03F05AEC04F0FDEC17F076EC29
:1017400009F06DEF08F0140E046E220EF66E310EE5
:10175000F76E000EF86E0900F550A0EC2CF0042E88
:10176000FAD744EC03F033EC0CF0FDEC17F08DEC01
:1017700009F06DEF08F0140E046E0E0EF66E310EC9
:10178000F76E000EF86E0900F550A0EC2CF0042E58
:10179000FAD744EC03F033EC0CF0FDEC17F0ADECB1
:1017A00009F06DEF08F0140E046EFA0EF66E300EAE
:1017B000F76E000EF86E0900F550A0EC2CF0042E28
:1017C000FAD744EC03F033EC0CF0FDEC17F0CAEC64
:1017D00009F06DEF08F0140E046EE60EF66E300E92
:1017E000F76E000EF86E0900F550A0EC2CF0042EF8
:1017F000FAD744EC03F033EC0CF0FDEC17F0E7EC17
:1018000009F06DEF08F0140E046EBE0EF66E300E89
:10181000F76E000EF86E0900F550A0EC2CF0042EC7
:10182000FAD744EC03F033EC0CF0FDEC17F004ECC9
:101830000AF06DEF08F0140E046ED20EF66E300E44
:10184000F76E000EF86E0900F550A0EC2CF0042E97
:10185000FAD744EC03F033EC0CF0FDEC17F021EC7C
:101860000AF06DEF08F026EC04F0010E75EC02F0C2
:1018700046EC04F01200140E046E8E0EF66E330E5B
:10188000F76E000EF86E0900F550A0EC2CF0042E57
:10189000FAD744EC03F06AEC04F0CEEC04F06DEF00
:1018A00008F0140E046EE20EF66E340EF76E000EA3
:1018B000F86E0900F550A0EC2CF0042EFAD744EC99
:1018C00003F067EC0CF06FEC0CF06DEF08F036EC09
:1018D00004F02A0E75EC02F046EC04F012004AEC1B
:1018E0000DF0D5EC1AF01AEC03F0080E036E1AECAA
:1018F00003F0A0EC2CF0032EFAD71200140E046EA5
:10190000F60EF66E340EF76E000EF86E0900F55006
:10191000A0EC2CF0042EFAD744EC03F094EC0CF07D
:101920009CEC0CF06DEF08F036EC04F02B0E75EC2F
:1019300002F046EC04F012004AEC0DF0D5EC1AF07F
:101940001AEC03F0080E036E1AEC03F0A0EC2CF076
:10195000032EFAD71200140E046E360EF66E310EF8
:10196000F76E000EF86E0900F550A0EC2CF0042E76
:10197000FAD744EC03F072EC04F0B2EC04F061EF3F
:1019800007F0140E046E4A0EF66E310EF76E000E5E
:10199000F86E0900F550A0EC2CF0042EFAD744ECB8
:1019A00003F002EC05F01AEC05F061EF07F0140EFD
:1019B000046E1A0EF66E340EF76E000EF86E090005
:1019C000F550A0EC2CF0042EFAD744EC03F00AEC0E
:1019D00005F036EC05F061EF07F0140E046E2E0EE4
:1019E000F66E340EF76E000EF86E0900F550A0EC9E
:1019F0002CF0042EFAD744EC03F012EC05F045EC81
:101A000005F061EF07F0140E046E5E0EF66E310EF7
:101A1000F76E000EF86E0900F550A0EC2CF0042EC5
:101A2000FAD744EC03F019EC0DF021EC0DF061EF66
:101A300007F036EC04F0050E75EC02F046EC04F00D
:101A400012003DEC0DF0F3EC02F0D5EC1AF0F3ECE3
:101A500002F0356E94EC2BF0300EA0EC2CF06D0EF5
:101A6000A0EC2CF0530EA0EC2CF0650EA0EC2CF0AA
:101A7000630EA0EC2CF061EF22F0DDEC02F0FE0A28
:101A8000FCE1F3EC02F0010AFCE1F3EC02F0F3EC10
:101A900002F0120004EC03F0FE0AFCE11AEC03F081
:101AA000010AFCE11AEC03F01AEC03F01200140E28
:101AB000046E720EF66E310EF76E000EF86E0900AF
:101AC000F550A0EC2CF0042EFAD744EC03F06DECAA
:101AD0000DF075EC0DF061EF07F036EC04F00D0E33
:101AE00075EC02F046EC04F012001CEC0BF0FF0A5F
:101AF000D8B41200D2EC02F00D0AD8A41200FDEC0A
:101B000017F0D2EC02F03B6EE8669EEF17F0A3EF01
:101B100017F0E7EC28F02CA83B702CA03B702CA40D
:101B200006D02CAA70EF07F0A4EC0DF0F2D736EC3B
:101B300004F00D0E75EC02F03B5075EC02F046EC33
:101B400004F01AEC23F0E5D7A00EB8EC2CF03B50D3
:101B5000E866EEEF2AF0FAEF2AF0140E046E860E15
:101B6000F66E310EF76E000EF86E0900F550A0EC1F
:101B70002CF0042EFAD744EC03F0C3EC0DF0CBECC0
:101B80000DF061EF07F036EC04F00E0E75EC02F08C
:101B900046EC04F012001CEC0BF0FF0AD8B4120063
:101BA000D2EC02F00E0AD8A41200FDEC17F0D2EC31
:101BB00002F03C6EE8669EEF17F0A3EF17F0E7EC3B
:101BC00028F02CA83C702CA03C702CA406D02CAA89
:101BD00070EF07F0FBEC0DF0F2D736EC04F00E0ED0
:101BE00075EC02F03C5075EC02F046EC04F01AEC97
:101BF00023F0DFEF0DF0A00EB8EC2CF03C50E866BF
:101C0000EEEF2AF0FAEF2AF0140E046E9A0EF66E3A
:101C1000310EF76E000EF86E0900F550A0EC2CF0B6
:101C2000042EFAD744EC03F07AEC04F078EC0AF0D6
:101C300061EF07F0140E046EAE0EF66E310EF76E05
:101C4000000EF86E0900F550A0EC2CF0042EFAD727
:101C500044EC03F082EC04F08CEC0AF061EF07F046
:101C6000140E046EC20EF66E310EF76E000EF86E94
:101C70000900F550A0EC2CF0042EFAD744EC03F048
:101C80008AEC04F0A0EC0AF061EF07F0140E046E89
:101C9000D60EF66E310EF76E000EF86E0900F55096
:101CA000A0EC2CF0042EFAD744EC03F092EC04F0F4
:101CB000B4EC0AF061EF07F0140E046EEA0EF66E53
:101CC000310EF76E000EF86E0900F550A0EC2CF006
:101CD000042EFAD744EC03F09AEC04F0C8EC0AF0B6
:101CE00061EF07F0140E046EFE0EF66E310EF76E05
:101CF000000EF86E0900F550A0EC2CF0042EFAD777
:101D000044EC03F0A2EC04F0DCEC0AF061EF07F025
:101D1000140E046E120EF66E320EF76E000EF86E92
:101D20000900F550A0EC2CF0042EFAD744EC03F097
:101D3000AAEC04F0F0EC0AF061EF07F0140E046E68
:101D4000260EF66E320EF76E000EF86E0900F55094
:101D5000A0EC2CF0042EFAD744EC03F0B4EC0EF017
:101D6000BCEC0EF061EF07F036EC04F0110E75ECF0
:101D700002F046EC04F012003DEC0DF0F3EC02F042
:101D8000D5EC1AF0F3EC02F0446E94EC2BF0300E2C
:101D9000A0EC2CF0530EA0EC2CF0650EA0EC2CF077
:101DA000630EA0EC2CF0200EA0EC2CF061EF22F0E2
:101DB000E7EC28F02CA8442A2CA044062CA406D03A
:101DC0002CAA70EF07F0F4EC0EF0F2D736EC04F02A
:101DD000110E75EC02F0445075EC02F046EC04F084
:101DE0001AEC23F0D8EF0EF0A00EB8EC2CF0445013
:101DF00094EC2BF0300EA0EC2CF0530EA0EC2CF059
:101E0000650EA0EC2CF0630EA0EC2CF0200EA0ECE4
:101E10002CF01200140E046E3A0EF66E320EF76EAF
:101E2000000EF86E0900F550A0EC2CF0042EFAD745
:101E300044EC03F020EC0FF028EC0FF061EF07F01A
:101E400036EC04F0120E75EC02F046EC04F01200D1
:101E50003DEC0DF0F3EC02F0940EB8EC2CF0140E07
:101E6000036E00EEC0F0F3EC02F0EE6EA0EC2CF08E
:101E7000032EF9D761EF22F010EEC0F085EC0FF0E1
:101E8000E7EC28F02CA854EC0FF02CA058EC0FF045
:101E90002CA26FEC0FF02CA67AEC0FF02CA40CD037
:101EA0002CAA70EF07F0ECD7E72A85EC0FF01200B0
:101EB000E70685EC0FF01200140E046E36EC04F009
:101EC000120E75EC02F000EEC0F0EE5075EC02F070
:101ED000042EFBD746EC04F01AEC23F0CDD7E12A10
:101EE000000EE222D40EE16202D010EEC0F085ECCA
:101EF0000FF01200E106000EE25ABF0EE16202D0BE
:101F000010EED3F085EC0FF01200940EB8EC2CF02C
:101F1000140E036E00EEC0F0EE50A0EC2CF0032E79
:101F2000FBD7930E046E140E036E00EEC0F0042A6D
:101F3000E250EA620AD0E150E96207D00450B8ECFE
:101F40002CF00E0EB8EC2CF01200EE50032EEFD752
:101F50001200140E046E4E0EF66E320EF76E000E68
:101F6000F86E0900F550A0EC2CF0042EFAD744ECE2
:101F700003F0BFEC0FF0C7EC0FF061EF07F036ECA9
:101F800004F0130E75EC02F046EC04F012003DEC88
:101F90000DF0D5EC1AF0F3EC02F0080E036E00EE33
:101FA0008CF0F3EC02F0EE6EA0EC2CF0032EF9D7DF
:101FB00061EF22F010EE8CF02DEC10F0E7EC28F041
:101FC0002CA8F2EC0FF02CA0FBEC0FF02CA217ECDD
:101FD00010F02CA622EC10F02CA416D02CAA70EF36
:101FE00007F0ECD7E72A5A0EE76402D0200EE76E1E
:101FF0002DEC10F01200E706200EE76002D05A0E1A
:10200000E76E2DEC10F01200140E046E36EC04F0A6
:10201000130E75EC02F000EE8CF0EE5075EC02F051
:10202000042EFBD746EC04F01AEC23F0C3D7E12AC8
:10203000000EE222940EE16202D010EE8CF02DEC44
:1020400010F01200E106000EE25A8B0EE16202D09F
:1020500010EE93F02DEC10F01200A00EB8EC2CF066
:10206000080E036E00EE8CF0EE50A0EC2CF0032E68
:10207000FBD79F0E046E080E036E00EE8CF0042A50
:10208000E250EA620AD0E150E96207D00450B8ECAD
:102090002CF00E0EB8EC2CF01200EE50032EEFD701
:1020A0001200140E046E620EF66E320EF76E000E03
:1020B000F86E0900F550A0EC2CF0042EFAD744EC91
:1020C00003F067EC10F06FEC10F061EF07F036EC06
:1020D00004F0140E75EC02F046EC04F012003DEC36
:1020E0000DF0D5EC1AF0F3EC02F0080E036E00EEE2
:1020F00094F0F3EC02F0EE6EA0EC2CF0032EF9D786
:1021000061EF22F010EE94F0D5EC10F0E7EC28F03F
:102110002CA89AEC10F02CA0A3EC10F02CA2BFEC91
:1021200010F02CA6CAEC10F02CA416D02CAA70EF3C
:1021300007F0ECD7E72A5A0EE76402D0200EE76ECC
:10214000D5EC10F01200E706200EE76002D05A0E20
:10215000E76ED5EC10F01200140E046E36EC04F0AD
:10216000140E75EC02F000EE94F0EE5075EC02F0F7
:10217000042EFBD746EC04F01AEC23F0C3D7E12A77
:10218000000EE2229C0EE16202D010EE94F0D5EC3B
:1021900010F01200E106000EE25A930EE16202D046
:1021A00010EE9BF0D5EC10F01200A00EB8EC2CF065
:1021B000080E036E00EE94F0EE50A0EC2CF0032E0F
:1021C000FBD79F0E046E080E036E00EE94F0042AF7
:1021D000E250EA620AD0E150E96207D00450B8EC5C
:1021E0002CF00E0EB8EC2CF01200EE50032EEFD7B0
:1021F0001200140E046E760EF66E320EF76E000E9E
:10220000F86E0900F550A0EC2CF0042EFAD744EC3F
:1022100003F00FEC11F017EC11F061EF07F036EC62
:1022200004F0150E75EC02F046EC04F012003DECE3
:102230000DF0D5EC1AF0F3EC02F0040E036E00EE94
:102240009CF0F3EC02F0EE6EA0EC2CF0032EF9D72C
:1022500051EC2BF061EF22F010EE9CF07FEC11F0CE
:10226000E7EC28F02CA844EC11F02CA04DEC11F078
:102270002CA269EC11F02CA674EC11F02CA416D051
:102280002CAA70EF07F0ECD7E72A5A0EE76402D0C9
:10229000200EE76E7FEC11F01200E706200EE760DB
:1022A00002D05A0EE76E7FEC11F01200040E046E9D
:1022B00036EC04F0150E75EC02F000EE9CF0EE50DA
:1022C00075EC02F0042EFBD746EC04F01AEC23F078
:1022D000C3D7E12A000EE222A00EE16202D010EE86
:1022E0009CF07FEC11F01200E106000EE25A9B0E0A
:1022F000E16202D010EE9FF07FEC11F01200A00E10
:10230000B8EC2CF0040E036E00EE9CF0EE50A0EC46
:102310002CF0032EFBD751EC2BF09F0E046E040E15
:10232000036E00EE9CF0042AE250EA620AD0E1500B
:10233000E96207D00450B8EC2CF00E0EB8EC2CF08B
:102340001200EE50032EEFD71200140E046E8A0E08
:10235000F66E320EF76E000EF86E0900F550A0EC26
:102360002CF0042EFAD744EC03F0BBEC11F0C3ECD4
:1023700011F061EF07F036EC04F0160E75EC02F088
:1023800046EC04F012003DEC0DF0D5EC1AF0F3EC45
:1023900002F0080E036E00EEA0F0F3EC02F0EE6E19
:1023A000A0EC2CF0032EF9D761EF22F010EEA0F094
:1023B00029EC12F0E7EC28F02CA8EEEC11F02CA0A0
:1023C000F7EC11F02CA213EC12F02CA61EEC12F07C
:1023D0002CA416D02CAA70EF07F0ECD7E72A5A0EDF
:1023E000E76402D0200EE76E29EC12F01200E70637
:1023F000200EE76002D05A0EE76E29EC12F01200B0
:10240000080E046E36EC04F0160E75EC02F000EEC9
:10241000A0F0EE5075EC02F0042EFBD746EC04F071
:102420001AEC23F0C3D7E12A000EE222A80EE162E3
:1024300004D010EEA0F029EC12F01200E106000E1C
:10244000E25A9F0EE16202D010EEA7F029EC12F0E2
:102450001200A00EB8EC2CF0080E036E00EEA0F0F7
:10246000EE50A0EC2CF0032EFBD79F0E046E080E4E
:10247000036E00EEA0F0042AE250EA620AD0E150B6
:10248000E96207D00450B8EC2CF00E0EB8EC2CF03A
:102490001200EE50032EEFD71200140E046E9E0EA3
:1024A000F66E320EF76E000EF86E0900F550A0ECD5
:1024B0002CF0042EFAD744EC03F063EC12F06BEC32
:1024C00012F061EF07F036EC04F0170E75EC02F035
:1024D00046EC04F012003DEC0DF0D5EC1AF0F3ECF4
:1024E00002F0080E036E00EEA8F0F3EC02F0EE6EC0
:1024F000A0EC2CF0032EF9D761EF22F010EEA8F03B
:10250000D1EC12F0E7EC28F02CA896EC12F02CA0FD
:102510009FEC12F02CA2BBEC12F02CA6C6EC12F031
:102520002CA416D02CAA70EF07F0ECD7E72A5A0E8D
:10253000E76402D0200EE76E29EC12F01200E706E5
:10254000200EE76002D05A0EE76ED1EC12F01200B6
:10255000080E046E36EC04F0170E75EC02F000EE77
:10256000A8F0EE5075EC02F0042EFBD746EC04F018
:102570001AEC23F0C3D7E12A000EE222B00EE1628A
:1025800002D010EEA8F0D1EC12F01200E106000E1D
:10259000E25AA70EE16202D010EEAFF0D1EC12F0D9
:1025A0001200A00EB8EC2CF0040E036E00EEA8F0A2
:1025B000EE50A0EC2CF0032EFBD79F0E046E080EFD
:1025C000036E00EEA8F0042AE250EA620AD0E1505D
:1025D000E96207D00450B8EC2CF00E0EB8EC2CF0E9
:1025E0001200EE50032EEFD71200140E046EB20E3E
:1025F000F66E320EF76E000EF86E0900F550A0EC84
:102600002CF0042EFAD744EC03F00BEC13F013EC8F
:1026100013F061EF07F036EC04F0180E75EC02F0E1
:1026200046EC04F012003DEC0DF0D5EC1AF0F3ECA2
:1026300002F0080E036E00EEB0F0F3EC02F0EE6E66
:10264000A0EC2CF0032EF9D761EF22F010EEB0F0E1
:1026500079EC13F0E7EC28F02CA83EEC13F02CA05A
:1026600047EC13F02CA263EC13F02CA66EEC13F0E5
:102670002CA416D02CAA70EF07F0ECD7E72A5A0E3C
:10268000E76402D0200EE76E79EC13F01200E70643
:10269000200EE76002D05A0EE76E79EC13F01200BC
:1026A000140E046E36EC04F0180E75EC02F000EE19
:1026B000B0F0EE5075EC02F0042EFBD746EC04F0BF
:1026C0001AEC23F0C3D7E12A000EE222B80EE16231
:1026D00002D010EEB0F079EC13F01200E106000E1B
:1026E000E25AAF0EE16202D010EEB7F079EC13F0CF
:1026F0001200A00EB8EC2CF0040E036E00EEB0F049
:10270000EE50A0EC2CF0032EFBD79F0E046E080EAB
:10271000036E00EEB0F0042AE250EA620AD0E15003
:10272000E96207D00450B8EC2CF00E0EB8EC2CF097
:102730001200EE50032EEFD71200140E046EC60ED8
:10274000F66E320EF76E000EF86E0900F550A0EC32
:102750002CF0042EFAD744EC03F0B3EC13F0BBECEE
:1027600013F061EF07F036EC04F0190E75EC02F08F
:1027700046EC04F012001CEC0BF0FF0AD8B4120077
:10278000B8EC02F0190AD8A4120000EE4DF0FDECEE
:1027900017F0B8EC02F0EE6EB8EC02F0EE6EB8ECAA
:1027A00002F0EE6ED6EC13F061EF07F0080E036E48
:1027B0004DC012F000EEB8F01236300ED8B0310E27
:1027C000EE6EA0EC2CF0032EF7D761EF22F0140E82
:1027D000046EDA0EF66E320EF76E000EF86E090019
:1027E000F550A0EC2CF0042EFAD744EC03F0FDECED
:1027F00013F005EC14F061EF07F036EC04F01A0E5C
:1028000075EC02F046EC04F012001CEC0BF0FF0A31
:10281000D8B41200B8EC02F01A0AD8A41200FDECE9
:1028200017F0B8EC02F0456EE8669EEF17F0A3EFE4
:1028300017F0140E046EEE0EF66E320EF76E000EEA
:10284000F86E0900F550A0EC2CF0042EFAD744ECF9
:1028500003F02FEC14F037EC14F061EF07F036ECD6
:1028600004F01B0E75EC02F046EC04F012001CECB8
:102870000BF0FF0AD8B41200B8EC02F01B0AD8A47F
:102880001200FDEC17F0B8EC02F0466EE8669EEF21
:1028900017F0A3EF17F0140E046E020EF66E330E4F
:1028A000F76E000EF86E0900F550A0EC2CF0042E27
:1028B000FAD744EC03F061EC14F069EC14F061EF2A
:1028C00007F036EC04F01C0E75EC02F046EC04F058
:1028D00012001CEC0BF0FF0AD8B41200B8EC02F0A6
:1028E0001C0AD8A41200FDEC17F0B8EC02F0476EF9
:1028F000E8669EEF17F0A3EF17F0140E046E160EA5
:10290000F66E330EF76E000EF86E0900F550A0EC6F
:102910002CF0042EFAD744EC03F093EC14F09BEC6B
:1029200014F061EF07F036EC04F01D0E75EC02F0C8
:1029300046EC04F012001CEC0BF0FF0AD8B41200B5
:10294000B8EC02F01D0AD8A41200FDEC17F0B8ECA8
:1029500002F0486EE8669EEF17F0A3EF17F0140E32
:10296000046E2A0EF66E330EF76E000EF86E090036
:10297000F550A0EC2CF0042EFAD744EC03F0C5EC93
:1029800014F0CDEC14F061EF07F036EC04F01E0EFD
:1029900075EC02F046EC04F012001CEC0BF0FF0AA0
:1029A000D8B41200B8EC02F01E0AD8A41200FDEC54
:1029B00017F0B8EC02F0496EE8669EEF17F0A3EF4F
:1029C00017F0140E046E3E0EF66E330EF76E000E08
:1029D000F86E0900F550A0EC2CF0042EFAD744EC68
:1029E00003F0F7EC14F0FFEC14F061EF07F036ECB5
:1029F00004F01F0E75EC02F046EC04F012001CEC23
:102A00000BF0FF0AD8B41200B8EC02F01F0AD8A4E9
:102A10001200FDEC17F0B8EC02F04A6EE8669EEF8B
:102A200017F0A3EF17F0140E046E520EF66E330E6D
:102A3000F76E000EF86E0900F550A0EC2CF0042E95
:102A4000FAD744EC03F029EC15F031EC15F061EF06
:102A500007F036EC04F0200E75EC02F046EC04F0C2
:102A600012001CEC0BF0FF0AD8B41200B8EC02F014
:102A7000200AD8A41200FDEC17F0B8EC02F04B6E5F
:102A8000E8669EEF17F0A3EF17F0140E046E660EC3
:102A9000F66E330EF76E000EF86E0900F550A0ECDE
:102AA0002CF0042EFAD744EC03F05BEC15F063EC49
:102AB00015F061EF07F036EC04F0210E75EC02F032
:102AC00046EC04F012001CEC0BF0FF0AD8B4120024
:102AD000B8EC02F0210AD8A41200FDEC17F0B8EC13
:102AE00002F04C6EE8669EEF17F0A3EF17F0140E9D
:102AF000046E7A0EF66E330EF76E000EF86E090055
:102B0000F550A0EC2CF0042EFAD744EC03F08DEC39
:102B100015F095EC15F061EF07F036EC04F0220E9D
:102B200075EC02F046EC04F012001CEC0BF0FF0A0E
:102B3000D8B41200B8EC02F0220AD8A41200FDECBE
:102B400017F0B8EC02F0506EE8669EEF17F0A3EFB6
:102B500017F0140E046EA20EF66E330EF76E000E12
:102B6000F86E0900F550A0EC2CF0042EFAD744ECD6
:102B700003F0BFEC15F0C7EC15F061EF07F036EC91
:102B800004F0230E75EC02F046EC04F012001CEC8D
:102B90000BF0FF0AD8B41200B8EC02F0230AD8A454
:102BA0001200FDEC17F0B8EC02F0516E72EC2CF054
:102BB0004EEC2BF0196A1200140E046EB60EF66E6F
:102BC000330EF76E000EF86E0900F550A0EC2CF0F5
:102BD000042EFAD744EC03F0F2EC15F0FAEC15F001
:102BE00061EF07F036EC04F0240E75EC02F046ECD1
:102BF00004F012001CEC0BF0FF0AD8B41200B8EC81
:102C000002F0240AD8A41200FDEC17F0B8EC02F090
:102C1000526EE8669EEF17F0A3EF17F0140E046EE5
:102C2000CA0EF66E330EF76E000EF86E0900F55000
:102C3000A0EC2CF0042EFAD744EC03F024EC16F0B0
:102C40002CEC16F061EF07F036EC04F0250E75EC75
:102C500002F046EC04F012001CEC0BF0FF0AD8B4B2
:102C60001200B8EC02F0250AD8A41200FDEC17F00F
:102C7000B8EC02F0536EE8669EEF17F0A3EF17F082
:102C8000140E046EDE0EF66E330EF76E000EF86E46
:102C90000900F550A0EC2CF0042EFAD744EC03F018
:102CA00056EC16F05EEC16F061EF07F036EC04F02F
:102CB000260E75EC02F046EC04F012001CEC0BF052
:102CC000FF0AD8B41200B8EC02F0260AD8A4120009
:102CD000FDEC17F0B8EC02F0546EE8669EEF17F0CA
:102CE000A3EF17F0140E046EF20EF66E330EF76EAD
:102CF000000EF86E0900F550A0EC2CF0042EFAD767
:102D000044EC03F088EC16F090EC16F061EF07F05D
:102D100036EC04F0270E75EC02F046EC04F01200DD
:102D20003DEC0DF0F3EC02F0940EB8EC2CF0140E28
:102D3000036E00EED4F0D2EC02F0EE6EA0EC2CF0BC
:102D4000032EF9D761EF22F010EED4F0EDEC16F07F
:102D5000E7EC28F02CA8BCEC16F02CA0C0EC16F088
:102D60002CA2D7EC16F02CA6E2EC16F02CA40CD07A
:102D70002CAA70EF07F0ECD7E72AEDEC16F0120062
:102D8000E706EDEC16F01200140E046E36EC04F0BB
:102D9000270E75EC02F000EED4F0EE5075EC02F068
:102DA000042EFBD746EC04F01AEC23F0CDD7E12A31
:102DB000000EE222E80EE16202D010EED4F0EDEC5B
:102DC00016F01200E106000EE25AD30EE16202D0C4
:102DD00010EEE7F0EDEC16F01200940EB8EC2CF0CB
:102DE000140E036E00EED4F0EE50A0EC2CF0032E87
:102DF000FBD7930E046E140E036E00EED4F0042A7B
:102E0000E250EA620AD0E150E96207D00450B8EC1F
:102E10002CF00E0EB8EC2CF01200EE50032EEFD773
:102E20001200140E046E060EF66E340EF76E000ECF
:102E3000F86E0900F550A0EC2CF0042EFAD744EC03
:102E400003F027EC17F02FEC17F061EF07F036ECEA
:102E500004F0280E75EC02F046EC04F012001CECB5
:102E60000BF0FF0AD8B41200B8EC02F0280AD8A47C
:102E70001200FDEC17F0B8EC02F0556EE866A3EF17
:102E800017F09EEF17F0E7EC28F02CA855702CA057
:102E900055702CA406D02CAA70EF07F05FEC17F049
:102EA000F2D736EC04F0280E75EC02F0555075ECB4
:102EB00002F046EC04F01AEC23F043EF17F0A00EFA
:102EC000B8EC2CF05550E866FAEF2AF0EEEF2AF055
:102ED00036EC04F02C0E75EC02F046EC04F01EEC1F
:102EE0002DF0C00EB8EC2CF0140E046E960EF66E9B
:102EF000350EF76E000EF86E0900F550A0EC2CF0C0
:102F0000042EFAD7120036EC04F0290E75EC02F00C
:102F100046EC04F01EEC2DF0C00EB8EC2CF0140EB4
:102F2000046E820EF66E350EF76E000EF86E090016
:102F3000F550A0EC2CF0042EFAD71200EEEC2AF09B
:102F4000196A61EF22F0FAEC2AF0196A61EF22F0B7
:102F5000530EA0EC2CF0700EA0EC2CF0610EA0EC47
:102F60002CF0630EA0EC2CF0650EA0EC2CF0200EE3
:102F7000A0EC2CF0200EA0EC2CF0200EA0EC2CF0FD
:102F8000196A12004C0EA0EC2CF0610EA0EC2CF093
:102F9000730EA0EC2CF0740EA0EC2CF0200EA0EC24
:102FA0002CF0480EA0EC2CF0440EA0EC2CF0520EAD
:102FB000A0EC2CF0196A12000650026E7E0E02245C
:102FC000D8B0FA2A3FEC1AF0A0EC2CF0062A042E16
:102FD000DCEF17F0E3EC2AF0D5EC1AF05EEC2BF006
:102FE0002CEC2BF061EF07F0E3EC2AF0E1EC2AF097
:102FF000D5EC1AF0040E026E1200E3EC2AF0D5ECC8
:103000001AF0080E026E1200E3EC2AF0940EB8ECEF
:103010002CF00E0EB8EC2CF0140E026E12004D6562
:103020006E752020202020202020202020202020FD
:103030002020446562756720496E666F202020203D
:103040002020202020205458204D792043616C6C92
:103050007369676E2020202020205458204D79204D
:1030600043616C6C7369676E3220202020205458B5
:103070002053746174696F6E2043616C6C7369676F
:103080006E20545820525054312043616C6C736947
:10309000676E202020205458205250543220436123
:1030A0006C6C7369676E20202020545820466C6138
:1030B000677320202020202020202020202052580C
:1030C000204D792043616C6C7369676E202020204D
:1030D00020205258204D792043616C6C7369676ED3
:1030E00032202020202052582053746174696F6E62
:1030F0002043616C6C7369676E20525820525054A3
:10310000312043616C6C7369676E20202020525817
:1031100020525054322043616C6C7369676E2020DA
:103120002020525820466C616773202020202020E8
:1031300020202020202054582044656C61792054A0
:10314000696D652020202020202054582054696D6E
:1031500065204F75742020202020202020205258E8
:10316000204B65657020416C6976652054696D65FA
:1031700020205258204175746F2E20506F6C617260
:10318000697479202020525820506F6C61726974E4
:1031900079202020202020202020545820506F6C9F
:1031A0006172697479202020202020202020434F44
:1031B0005320436865636B2020202020202020209E
:1031C000202043524320436865636B202020202049
:1031D0002020202020204C617374204672616D6590
:1031E0002073656E6420202020204865616465722C
:1031F0002047656E65726174696F6E202020486596
:10320000616465722047656E2E20547970652020B8
:10321000202048616C662F46756C6C204455504CDC
:10322000455820202020426561636F6E20496E74EE
:10323000657276616C54696D6572426561636F6E2B
:10324000204D6573736167652020202020204D7913
:103250002052657065617465722043616C6C73699E
:10326000676E416C746572204D792043616C6C739C
:1032700069676E202020416C746572204D7920436F
:10328000616C6C7369676E322020416C74657220CA
:10329000596F75722043616C6C7369676E20416C65
:1032A00074657220525054312043616C6C736967AD
:1032B0006E20416C74657220525054322043616C10
:1032C0006C7369676E20416C74657220466C61672F
:1032D00073202020202020202020526570656174FA
:1032E00065722043616C6C20436865636B20526596
:1032F0007065617465722044757020436865636B06
:103300002020526570656174657220447570204399
:103310006C6561722020416C746572204D79204388
:10332000616C6C20536574202020416C74657220A0
:103330004D792043616C6C32205365742020416CC0
:1033400074657220596F75722043616C6C205365EF
:103350007420416C74657220525054312043616C6A
:103360006C2053657420416C746572205250543245
:103370002043616C6C2053657420416C746572202D
:10338000466C6167732053657420202020205049CB
:10339000432056657273696F6E2020202020202004
:1033A00020204469676974616C20436F6465202044
:1033B0002020202020204469676974616C20436FBD
:1033C000646520536574202020204265666F726515
:1033D00020496E73657274202020202020204166D1
:1033E00074657220496E736572742020202020203D
:1033F0002020496E73657274204D65737361676533
:10340000202020202020555342204F6E2F4F6666EB
:10341000202020202020202020204A6974746572FA
:10342000204275666665722073697A652020532F85
:103430004E20537175656C63682056616C7565200C
:1034400020205258204175746F2E20506F6C61728D
:10345000697479202020525820506F6C6172697411
:1034600079202020202020202020545820506F6CCC
:103470006172697479202020202020202020547837
:103480002044656C61792054696D652020202020DE
:103490002020475053204D657373616765202020BD
:1034A00020202020202055706461746520537563AE
:1034B000636573732020202020205570646174653B
:1034C000204661696C20202020202020202055707B
:1034D00064617465204D6F646520202020202020C9
:1034E0002020557365722049442020202020202070
:1034F00020202020202053657269616C204E756D5C
:1035000062657220202020202020446973706C6145
:10351000792053657474696E6720202020204750FD
:1035200053204D657373616765204F4E2F4F46469C
:1035300020202A2A2A204E6F20486973746F7279DE
:10354000202A2A2A20202A2A204C6174657374209C
:103550005265636F7264202A2A202A2A2A204C612D
:103560007374205265636F7264202A2A2A204E6F7A
:103570007420436F6E6E656374204E6F64652041E6
:1035800064614E6F6465204164617074657220529D
:103590006573657420204E6F64652041642E204958
:1035A0006E69742E205265736574940EB8EC2CF01D
:1035B0000C0E036ED00EF66E350EF76E000EF86E22
:1035C0000900F550A0EC2CF0032EE0EF1AF01200E9
:1035D0004375722E2056616C75653A20FF0E1A6E87
:1035E0001C2E61EF22F01A6A1B6A61EF22F01A06A4
:1035F00061EF22F09BEC02F0136EFE0A05E1195018
:10360000020A02E161EF22F0195001E10ED0E84E0A
:1036100013D0E84E18D0E84E21D0E84E26D0E84E20
:1036200040D0E84EFFD061EF22F01350FE0AD8A43C
:1036300061EF22F0192A12001350FE0AD8A461EF9C
:1036400022F0192A12001350FE0AD8B412001350A7
:10365000010AD8A461EF22F0192A120013507F0A40
:10366000D8A461EF22F0192A120013501D0A02E1BA
:10367000192A12001350FA0AD8B4B0D71350FB0A13
:10368000D8B4F7EF1AF01350200AD8A403D0060ECE
:10369000196E120013501C0AD8A461EF22F042EFF9
:1036A0001CF0000EFB6E360EFA6E13380F0BE84658
:1036B000E846036EC20E0326000EFA22FB220350D8
:1036C000F96E81EF1BF061EF22F061EF22F061EF04
:1036D00022F061EF22F061EF22F061EF22F061EF62
:1036E00022F061EF22F061EF22F061EF22F061EF52
:1036F00022F0B1EF1BF0E1EF1BF061EF22F061EF80
:1037000022F0000EFB6E370EFA6E13500F0BE846D8
:10371000E846036E220E0326000EFA22FB22035017
:10372000F96EB7EF1CF061EF22F061EF22F068EF65
:103730001DF07AEF1DF05AEF1EF061EF22F061EFFD
:1037400022F061EF22F061EF22F061EF22F061EFF1
:1037500022F061EF22F061EF22F061EF22F061EFE1
:1037600022F0000EFB6E370EFA6E13500F0BE84678
:10377000E846036E820E0326000EFA22FB22035057
:10378000F96EB5EF1EF061EF22F061EF22F061EF0C
:1037900022F061EF22F061EF22F061EF22F061EFA1
:1037A00022F061EF22F061EF22F061EF22F061EF91
:1037B00022F061EF22F061EF22F061EF22F061EF81
:1037C00022F0000EFB6E370EFA6E13500F0BE84618
:1037D000E846036EE20E0324D8B0FA2AD8B0FB2ADA
:1037E000F96E61EF22F061EF22F061EF22F061EFFC
:1037F00022F061EF22F061EF22F061EF22F061EF41
:1038000022F061EF22F061EF22F061EF22F0F5EF9C
:1038100021F03FEF22F061EF22F061EF22F061EF43
:1038200022F01200000EFB6E380EFA6E13500F0BD2
:10383000E846E846036E440E0324D8B0FA2AD8B00E
:10384000FB2AF96E49EF1CF061EF22F061EF22F0E4
:1038500061EF22F061EF22F061EF22F061EF22F0E0
:1038600061EF22F061EF22F061EF22F061EF22F0D0
:1038700061EF22F061EF22F061EF22F061EF22F0C0
:10388000D0EF22F0B8EC02F0136E01E154D061EFFA
:1038900022F0090E026ED2EC02F0022EFCD70A0EC4
:1038A0002A6ED2EC02F00101546FD2EC02F0556F97
:1038B000D2EC02F0566FD2EC02F0386ED2EC02F08D
:1038C000396E550E546309D02D0E556306D0160E71
:1038D000566303D0576B61EF22F0550E546308D046
:1038E000550E556305D0550E566302D061EF22F098
:1038F000572B57A110D054C14EF1700E4E1B55C11D
:103900004FF14F0E4F1B56C150F1930E501B22EC3E
:103910002CF061EF22F054C151F1700E511B55C1D2
:1039200052F14F0E521B56C153F1930E531B22EC12
:103930002CF0B5EF1EF0A60EB8EC2CF0B8EC02F0AF
:10394000000F200ED8A42A0EA0EC2CF061EF22F07C
:1039500007A6000C15EC2DF015EC2DF007A6000CB9
:1039600015EC2DF015EC2DF007A6000C010C0890BD
:10397000B8EC02F0186E070B1BE118C015F01EEC36
:103980002DF0900EB8EC2CF0440E15BC520EA0ECAD
:103990002CF04E0E15BA420EA0EC2CF0440E15B8C9
:1039A000430EA0EC2CF04E0E15B6450EA0EC2CF0FC
:1039B000CC0EB8EC2CF018C013F0070E1316000E46
:1039C00004E0080F132EE1EF1CF0066E080E026EE5
:1039D000000EF86E3A0EF76E900EF66E0650F62652
:1039E000000EF722F8220900F550A0EC2CF0022E70
:1039F000FAD71850070BD8A461EF22F015EC04F0A9
:103A00009BEC1EF061EF22F01EEC2DF0240E026EF6
:103A100001EE00F0200EEE1803E1022EFBD712009B
:103A2000900EB8EC2CF0440E15BC520EA0EC2CF00D
:103A30004E0E15BA420EA0EC2CF0440E15B8430EF3
:103A4000A0EC2CF04E0E15B6450EA0EC2CF0CC0ED2
:103A5000B8EC2CF018C013F0070E1316000E03E09C
:103A6000080F132EFDD7066E080E026E000EF86EBC
:103A70003A0EF76E900EF66E0650F626000EF722FE
:103A8000F8220900F550A0EC2CF0022EFAD7120013
:103A9000202020204E554C4C52656C617920556E8B
:103AA0004E6F2052656C6179202020202041434BCD
:103AB0002020526573656E642020556E75736564B1
:103AC0004175746F20526570202020204E554C4C5B
:103AD000800EB8EC2CF0080E046EA8EC1CF0000F61
:103AE000D8A461EF22F09BEC02F0A0EC2CF0042EA5
:103AF0006DEF1DF0200E036E01EE6CF0D2EC02F0C3
:103B0000EE6E032EFBD7080E036E01EE74F021EE6D
:103B100084F0EE50DE6204D0032EFBD761EF22F07A
:103B2000E8C0EAFFE9C0E9FFB2EC22F0200E036E24
:103B300021EE6CF0DECFEEFF032EFCD70F0EEA185D
:103B4000D8A408D005EE00F0EACFEAF0E9CFEBF018
:103B5000568006D056A004D0EACFEAF0E9CFEBF0C9
:103B6000EACFE8F0E9CFE9F000D0060EB8EC2CF08F
:103B700021EE6CF008A0BFEF1DF0E1EC2AF0940EEE
:103B8000B8EC2CF0080E046E01EE08F015BC01EE46
:103B900000F0DE50EE6E1FB000D0A0EC2CF0042E32
:103BA000F8D79E0EB8EC2CF0080E046E01EE00F073
:103BB00015BC01EE08F0DE50EE6E1FB000D0A0EC98
:103BC0002CF0042EF8D7C00EB8EC2CF0080E046EC2
:103BD00001EE18F0DE50EE6EA0EC2CF0042EEAEFB1
:103BE0001DF0800EB8EC2CF0080E046E01EE10F003
:103BF000DE50EE6EA0EC2CF0042EF8EF1DF061EF1D
:103C000022F09E0EB8EC2CF0080E046E01EE08F0C7
:103C100015BC01EE00F0EE50A0EC2CF0042EFBD70A
:103C2000940EB8EC2CF0080E046E01EE00F015BCFA
:103C300001EE08F0EE50A0EC2CF0042EFBD7C00EE5
:103C4000B8EC2CF0080E046E01EE18F0EE50A0EC6B
:103C50002CF0042E26EF1EF0800EB8EC2CF0080E8F
:103C6000046E01EE10F0EE50A0EC2CF0042EFBD709
:103C7000120001EE10F011EE34F0080E026EEECFDD
:103C8000E6FF022EFCD7120001EE00F011EE24F048
:103C9000100E026EEECFE6FF022EFCD7120001EEF0
:103CA00008F011EE2CF0080E026EEECFE6FF022EA9
:103CB000FCD712009E0EB8EC2CF0080E046EA8EC97
:103CC0001CF0000FD8A461EF22F09BEC02F0A0ECF6
:103CD0002CF0042E5FEF1EF0940EB8EC2CF0080EC2
:103CE000046EA8EC1CF0000FD8A461EF22F09BEC4E
:103CF00002F0A0EC2CF0042E71EF1EF0C00EB8EC18
:103D00002CF0080E046EA8EC1CF0000FD8A461EF94
:103D100022F09BEC02F0A0EC2CF0042E83EF1EF0BE
:103D200061EF22F004EC1DF001EC1EF020EC22F01B
:103D30009BEC1EF01200140E046E01EE58F0200EE3
:103D4000EE1804E1042EFBD72A6A1200D40EB8EC58
:103D50002CF0140E046E01EE58F0EE50A0EC2CF096
:103D6000042EFBD7050E2A6E120001EE4EF0EE5027
:103D7000136E660AD8B461EF22F01FA004D013506E
:103D8000F00B300A66E0060E08A0B8EC2CF01350D9
:103D9000400AD8A414D0D40E08A0B8EC2CF0050E1C
:103DA000046E21EE58F0EE50DE6E08A0A0EC2CF070
:103DB000042EF9D71E0E2A6E576B61EF22F01350B6
:103DC000410AD8A414D0D90E08A0B8EC2CF0050EE6
:103DD000046E21EE5DF0EE50DE6E08A0A0EC2CF03B
:103DE000042EF9D71E0E2A6E576B61EF22F0135086
:103DF000420AD8A414D0DE0E08A0B8EC2CF0050EB0
:103E0000046E21EE62F0EE50DE6E08A0A0EC2CF005
:103E1000042EF9D71E0E2A6E576B61EF22F0135055
:103E2000430AD8A461EF22F0E30E08A0B8EC2CF00E
:103E3000050E046E21EE67F0EE50DE6E08A0A0ECD9
:103E40002CF0042E1CEF1FF01E0E2A6E576B61EF34
:103E500022F013500F0B046E050E0460046E000177
:103E60008151B8EC2CF00880EE50136E240A08E162
:103E7000010E0001804D04D0806B802BEBEF20F011
:103E8000000EFB6E3E0EFA6E00018051E846E846D9
:103E9000036EA00E0326000EFA22FB220350F96ED9
:103EA000EBEF20F098EF1FF0A6EF1FF0AFEF1FF041
:103EB000C1EF1FF0D4EF1FF0DDEF1FF0EEEF1FF0AA
:103EC000F6EF1FF024EF20F04BEF20F062EF20F030
:103ED00067EF20F06FEF20F077EF20F07FEF20F01A
:103EE00087EF20F09BEF20F0B8EF20F0CAEF20F032
:103EF000FCEF20F004EF21F00CEF21F022EF21F095
:103F000044EF21F053EF21F05AEF21F06CEF21F054
:103F100073EF21F079EF21F082EF21F098EF21F09B
:103F2000CCEF21F0D4EF21F0E7EF21F0EFEF21F01B
:103F30001350470A03E10001802B4DD11350240A8E
:103F4000D8A4EAEF20F00C0E806F45D11350500A30
:103F5000D8A4EAEF20F00001802BEBEF20F0135003
:103F6000470AD8A404D00001802BEBEF20F01350B7
:103F7000520AD8A4EAEF20F0140E0001806FEBEF94
:103F800020F013504C0AD8A4CAEF1FF00001802B78
:103F9000EBEF20F01350470AD8A4EAEF20F01D0EF3
:103FA0000001806FEBEF20F013504C0AD8A4EAEF29
:103FB00020F00001802BEBEF20F013502C0AD8A446
:103FC000EBEF20F00001802B940E816FB8EC2CF009
:103FD000200EA0EC2CF0812BEBEF20F013502C0ADC
:103FE000D8A43AD00001802BEBEF20F013502C0A1C
:103FF000D8A42CEF20F0080E056E200EA0EC2CF0BB
:10400000052EFBD70001802BD40E816FB8EC2CF06D
:10401000EBEF20F08251050AD8B4EAEF20F01350FC
:10402000A0EC2CF00001812B822B8251020AD8B423
:104030001FEF20F08251040AD8A4EBEF20F03A0ED3
:10404000A0EC2CF0812BC7D013502C0AD8A42CEF55
:1040500020F0802BEBEF20F01350A0EC2CF0812B04
:10406000BAD01350A0EC2CF0812BE20E811908E19C
:104070008151B8EC2CF0200EA0EC2CF0812BABD0B1
:10408000E50E811907E18151B8EC2CF03A0EA0EC55
:104090002CF0812BA0D013502C0AD8A42CEF20F0A8
:1040A000A70EB8EC2CF0470EA0EC2CF0802BDF0E06
:1040B000816FB8EC2CF0200EA0EC2CF0812B826BE1
:1040C000EBEF20F013502C0AD8B484D0A3D71350B0
:1040D000430AD8A4EAEF20F0802BEBEF20F0135036
:1040E000520AD8A4EAEF20F0802BEBEF20F0135017
:1040F000430AD8A4EAEF20F0802BEBEF20F0135016
:104100003A0AD8A4EBEF20F0802BEBEF20F013500D
:104110002F0AD8B4802BA70EB8EC2CF0470EA0ECD9
:104120002CF0DF0E816FB8EC2CF0200EA0EC2CF000
:10413000812B826B50D013507A0A0AE01350680A20
:1041400090E1E20EB8EC2CF03A0EA0EC2CF006D088
:10415000E20EB8EC2CF02F0EA0EC2CF0802B940E7D
:10416000816FB8EC2CF0200EA0EC2CF0812B33D01A
:1041700013502F0AD8A42CEF20F0080E056E200E45
:10418000A0EC2CF0052EFBD7802BD40E816FB8EC61
:104190002CF021D01350450AD8B406D01350570A3A
:1041A000D8B402D02CEF20F01350A0EC2CF0200E4D
:1041B000A0EC2CF0200EA0EC2CF0200EA0EC2CF0AB
:1041C000EAEF20F09F0E816FB8EC2CF04EEC2BF054
:1041D00051EC2BF0806BA80E816703D0A70E816F86
:1041E00006D0E80E816703D0E70E816F00D0042E61
:1041F00034EF1FF061EF22F013504D0AD8A4EAEF1C
:1042000020F0802BEBEF20F01350430AD8A4EAEF04
:1042100020F0802BEBEF20F013502C0AD8A4EAEF0B
:1042200020F0A70EB8EC2CF0470EA0EC2CF0802B61
:10423000DF0E816FB8EC2CF0200EA0EC2CF0812B5F
:10424000EBEF20F013502C0AD8A42AEF21F0802B9A
:10425000EBEF20F01350A0EC2CF0812BE20E811933
:1042600008E18151B8EC2CF03A0EA0EC2CF0812B37
:10427000B2D7E50E8119AFE18151B8EC2CF03A0EBE
:10428000A0EC2CF0812BA7D713502C0AD8A4EBEF6D
:1042900020F0802B940E816FB8EC2CF0200EA0EC57
:1042A0002CF0812B98D713502C0AD8A42CEF20F097
:1042B000802B91D713502C0AD8A42CEF20F0802B00
:1042C000080E056E200EA0EC2CF0052EFBD7D40EA8
:1042D000816FB8EC2CF07FD713502C0AD8A42CEFA8
:1042E00020F0802B78D713502C0AD8A42CEF20F084
:1042F00071D71350410AD8A4EAEF20F0802B08822E
:10430000EBEF20F013502C0AD8A4EAEF20F0A70E10
:10431000B8EC2CF0470EA0EC2CF0802BDF0E816F58
:10432000B8EC2CF0200EA0EC2CF0812BEBEF20F061
:1043300013502C0AD8A4A9EF21F0802B940E816F82
:10434000B8EC2CF0200EA0EC2CF0812B0892EBEFB7
:1043500020F013502E0AD8B40892135008B2A0ECE3
:104360002CF0812BE20E811909E18151B8EC2CF07F
:104370003A0EA0EC2CF0812BEBEF20F0E50E81192A
:10438000D8A4EBEF20F08151B8EC2CF03A0EA0EC61
:104390002CF0812BEBEF20F013502C0AD8A42CEF3B
:1043A00020F0802BEBEF20F013502C0AD8A42CEF38
:1043B00020F0802B080E056E200EA0EC2CF0052EB0
:1043C000FBD7D40E816FB8EC2CF0EBEF20F013503C
:1043D0002C0AD8A42CEF20F0802BEBEF20F0135008
:1043E0002C0AD8A42CEF20F0F5D61850070B68E162
:1043F000880EB8EC2CF0200EA0EC2CF0078A040EEE
:10440000046E01EE20F0A8EC1CF0000FD8A460EFC1
:1044100022F09BEC02F0EE6E136EA0EC2CF0135029
:10442000200AD8A4079A042EEED707BA60EF22F02C
:10443000880EB8EC2CF02F0EA0EC2CF060EF22F0E0
:10444000880EB8EC2CF0200EA0EC2CF0078A040E9D
:10445000046E01EE20F0EE50136EA0EC2CF0135021
:10446000200AD8A4079A042E2BEF22F007BA1200D4
:10447000880EB8EC2CF02F0EA0EC2CF01200880E59
:10448000B8EC2CF0200EA0EC2CF0078A040E046E81
:10449000A8EC1CF0000FD8A461EF22F09BEC02F016
:1044A000136EA0EC2CF01350200AD8A4079A042E07
:1044B00048EF22F007BA61EF22F0880E19EF22F0E0
:1044C000079C196A1200A70EB8EC2CF0200EA0EC85
:1044D0002CF0C80EB8EC2CF0200EA0EC2CF0200E26
:1044E000A0EC2CF0200EA0EC2CF0200EA0EC2CF078
:1044F00007A81EEC2DF0DF0EB8EC2CF0200EA0EC7F
:104500002CF0020E52EC29F0126E1238030B300917
:10451000A0EC2CF012500F0B3009A0EC2CF03A0E4E
:10452000A0EC2CF0010E52EC29F0126E1238070BA1
:104530003009A0EC2CF012500F0B3009A0EC2CF03D
:104540003A0EA0EC2CF0000E52EC29F0126E12384C
:10455000070B3009A0EC2CF012500F0B3009A0EC27
:104560002CF01200020E52EC29F03F0BEE6E010E01
:1045700052EC29F07F0BEE6E000E52EC29F07F0B0F
:10458000EE6E060E52EC29F0EE6E050E52EC29F09E
:104590001F0BEE6E040E52EC29F03F0BEE6E120074
:1045A00001EE3CF0080E026E9BEC02F0EE6E022E65
:1045B000FBD7200EEE6EEE6E080E026E9BEC02F044
:1045C000EE6E022EFBD7A4EC28F063EC22F0120072
:1045D000E7EC28F02CA8332A2CA033062CA406D014
:1045E0002CAA70EF07F004EC23F0F2D736EC04F0BD
:1045F000030E75EC02F0335075EC02F046EC04F05B
:104600001AEC23F0E8EF22F0A00EB8EC2CF03350B7
:1046100094EC2BF0300EA0EC2CF06D0EA0EC2CF0F6
:10462000530EA0EC2CF0650EA0EC2CF0630EA0EC69
:104630002CF01200D40EB8EC2CF03DEC0DF0FB0A7F
:104640000FE0140E046EBA0EF66E340EF76E000E06
:10465000F86E0900F550A0EC2CF0042EFAD71200E9
:10466000140E046EA60EF66E340EF76E000EF86E83
:104670000900F550A0EC2CF0042EFAD71200E7EC5C
:1046800028F02CA8342A2CA034062CA406D02CAA5E
:1046900070EF07F05BEC23F0F2D736EC04F0040E79
:1046A00075EC02F0345075EC02F046EC04F01AECB4
:1046B00023F03FEF23F0A00EB8EC2CF0345094EC34
:1046C0002BF0300EA0EC2CF0530EA0EC2CF0650E6D
:1046D000A0EC2CF0630EA0EC2CF0200EA0EC2CF043
:1046E0001200E7EC28F02CA8352A2CA035062CA4C3
:1046F00006D02CAA70EF07F08DEC23F0F2D736EC41
:1047000004F0050E75EC02F0345075EC02F046EC46
:1047100004F01AEC23F071EF23F0A00EB8EC2CF0AB
:10472000355094EC2BF0300EA0EC2CF06D0EA0EC7C
:104730002CF0530EA0EC2CF0650EA0EC2CF0630EC8
:10474000A0EC2CF01200E7EC28F02CB80AD0372AA5
:10475000000E3622040E361804E1375002E1366AA4
:10476000376A2CB009D03706000E365AD8B004D0BC
:10477000030E366EFF0E376E2CA406D02CAA70EFF7
:1047800007F0DFEC23F0DFD7060E036ED89036C0BB
:1047900013F037C014F014361336032EFCD736EC62
:1047A00004F0080E75EC02F0135075EC02F0145092
:1047B00075EC02F046EC04F01AEC23F0C4D7A00E1E
:1047C000B8EC2CF0DCEC2BF01200E7EC28F02CA875
:1047D0003A2A2CA03A062CA406D02CAA70EF07F097
:1047E00000EC24F0F2D736EC04F0090E75EC02F080
:1047F0003A5075EC02F046EC04F01AEC23F0E5D7E1
:10480000A00EB8EC2CF03A505EEC2BF01200E7EC66
:1048100028F02CA83D702CA03D702CA406D02CAA0A
:1048200070EF07F022EC24F0F2D736EC04F00F0E14
:1048300075EC02F03D5075EC02F046EC04F01AEC19
:1048400023F0E5D7A00EB8EC2CF03D50E866EEEF73
:104850002AF0FAEF2AF0E7EC28F02CA83E702CA002
:104860003E702CA406D02CAA70EF07F046EC24F082
:10487000F2D736EC04F00C0E75EC02F03E5075ECFD
:1048800002F046EC04F01AEC23F0E5D7A00EB8ECE9
:104890002CF03E50E866EEEF2AF0FAEF2AF0E7EC53
:1048A00028F02CA83F702CA03F702CA406D02CAA76
:1048B00070EF07F06AEC24F0F2D736EC04F00A0E41
:1048C00075EC02F03F5075EC02F046EC04F01AEC87
:1048D00023F0E5D7A00EB8EC2CF03F50E866EEEFE1
:1048E0002AF0FAEF2AF0E7EC28F02CA840702CA070
:1048F00040702CA406D02CAA70EF07F08EEC24F0A8
:10490000F2D736EC04F00B0E75EC02F0405075EC6B
:1049100002F046EC04F01AEC23F0E5D7A00EB8EC58
:104920002CF04050E866EEEF2AF0FAEF2AF0E7ECC0
:1049300028F02CA841702CA041702CA406D02CAAE1
:1049400070EF07F0B3EC24F0F2D736EC04F0070E6A
:1049500075EC02F0415075EC02F046EC04F01AECF4
:1049600023F097EF24F0A00EB8EC2CF04150E8664D
:10497000EEEF2AF0FAEF2AF0E7EC28F02CA84270CC
:104980002CA042702CA406D02CAA70EF07F0D8EC13
:1049900024F0F2D736EC04F0060E75EC02F042502B
:1049A00075EC02F046EC04F01AEC23F0BCEF24F0B6
:1049B000A00EB8EC2CF04250E866E1EF24F0E5EFF1
:1049C00024F0A8EC17F061EF22F0C2EC17F061EFD1
:1049D00022F0E7EC28F02CA843702CA043702CA404
:1049E00006D02CAA70EF07F005EC25F0F2D736ECD4
:1049F00004F0100E75EC02F0435075EC02F046EC3A
:104A000004F01AEC23F0E9EF24F0A00EB8EC2CF03F
:104A10004350E8661AEF2BF00AEF2BF010EEB8F0D7
:104A20005CEC25F0E7EC28F02CA880EC25F02CA01D
:104A300080EC25F02CA246EC25F02CA651EC25F0BC
:104A40002CA404D02CAA70EF07F0ECD7080E046E4B
:104A500000EEB8F0D890300EEE62D8801236042EF8
:104A6000F9D712C04DF0030E046E36EC04F0190EA7
:104A700075EC02F000EE4DF0EE5075EC02F0042EF5
:104A8000FBD746EC04F01AEC23F0C8D7E12A000E5D
:104A9000E222C00EE16202D010EEB8F05CEC25F02C
:104AA0001200E106000EE25AB70EE16202D010EEEB
:104AB000BFF05CEC25F01200A00EB8EC2CF0080E54
:104AC000036E00EEB8F0EE50A0EC2CF0032EFBD7F6
:104AD0009F0E046E080E036E00EEB8F0042AE2503A
:104AE000EA620AD0E150E96207D00450B8EC2CF039
:104AF0000E0EB8EC2CF01200EE50032EEFD7120081
:104B0000300EE76201D0310EE76E5CEC25F012004A
:104B1000E7EC28F02CA845702CA045702CA406D0FA
:104B20002CAA70EF07F0A4EC25F0F2D736EC04F0D5
:104B30001A0E75EC02F0455075EC02F046EC04F0EC
:104B40001AEC23F088EF25F0A00EB8EC2CF04550BD
:104B5000E866EEEF2AF0FAEF2AF0E7EC28F02CA84E
:104B600046702CA046702CA406D02CAA70EF07F03B
:104B7000C9EC25F0F2D736EC04F01B0E75EC02F010
:104B8000465075EC02F046EC04F01AEC23F0ADEF61
:104B900025F0A00EB8EC2CF04650E866EEEF2AF0B7
:104BA000FAEF2AF0E7EC28F02CA847702CA0477009
:104BB0002CA406D02CAA70EF07F0EEEC25F0F2D76B
:104BC00036EC04F01C0E75EC02F0475075EC02F068
:104BD00046EC04F01AEC23F0D2EF25F0A00EB8EC6E
:104BE0002CF04750E866EEEF2AF0FAEF2AF0E7ECF7
:104BF00028F02CA848702CA048702CA406D02CAA11
:104C000070EF07F013EC26F0F2D736EC04F01D0E2F
:104C100075EC02F0485075EC02F046EC04F01AEC2A
:104C200023F0D2EF25F0A00EB8EC2CF04850E86647
:104C3000EEEF2AF0FAEF2AF0E7EC28F02CA8497002
:104C40002CA049702CA406D02CAA70EF07F038ECE9
:104C500026F0F2D736EC04F01E0E75EC02F0495047
:104C600075EC02F046EC04F01AEC23F0D2EF25F0DC
:104C7000A00EB8EC2CF04950E866EEEF2AF0FAEFFF
:104C80002AF0E7EC28F02CA84A702CA04A702CA43B
:104C900006D02CAA70EF07F05DEC26F0F2D736ECC8
:104CA00004F01F0E75EC02F04A5075EC02F046EC71
:104CB00004F01AEC23F0D2EF25F0A00EB8EC2CF0A3
:104CC0004A50E866EEEF2AF0FAEF2AF0E7EC28F017
:104CD0002CA84B702CA04B702CA406D02CAA70EFE3
:104CE00007F082EC26F0F2D736EC04F0200E75ECDB
:104CF00002F04B5075EC02F046EC04F01AEC23F095
:104D0000D2EF25F0A00EB8EC2CF04B50E866EEEF99
:104D10002AF0FAEF2AF0E7EC28F02CA84C702CA02F
:104D20004C702CA406D02CAA70EF07F0A7EC26F04C
:104D3000F2D736EC04F0210E75EC02F04C5075EC15
:104D400002F046EC04F01AEC23F0D2EF25F0A00EAE
:104D5000B8EC2CF04C50E866EEEF2AF0FAEF2AF0AF
:104D6000E7EC28F02CA850702CA050702CA406D092
:104D70002CAA70EF07F0CCEC26F0F2D736EC04F05A
:104D8000220E75EC02F0505075EC02F046EC04F087
:104D90001AEC23F0B0EF26F0A00EB8EC2CF0505037
:104DA000E866EEEF2AF0FAEF2AF0E7EC28F02CA8FC
:104DB000512A2CA051062CA406D02CAA70EF07F083
:104DC000F1EC26F0F2D736EC04F0230E75EC02F08D
:104DD000515075EC02F046EC04F01AEC23F0D5EFDC
:104DE00026F0A00EB8EC2CF0515072EC2CF04EECEA
:104DF0002BF0196A1200E7EC28F02CA852702CA0B6
:104E000052702CA406D02CAA70EF07F017EC27F0F4
:104E1000F2D736EC04F0240E75EC02F0525075EC2B
:104E200002F046EC04F01AEC23F0FBEF26F0A00EA3
:104E3000B8EC2CF05250E866EEEF2AF0FAEF2AF0C8
:104E4000E7EC28F02CA853702CA053702CA406D0AB
:104E50002CAA70EF07F03CEC27F0F2D736EC04F008
:104E6000250E75EC02F0535075EC02F046EC04F0A0
:104E70001AEC23F020EF27F0A00EB8EC2CF05350E2
:104E8000E866EEEF2AF0FAEF2AF0E7EC28F02CA81B
:104E900054702CA054702CA406D02CAA70EF07F0EC
:104EA00061EC27F0F2D736EC04F0260E75EC02F038
:104EB000545075EC02F046EC04F01AEC23F045EF88
:104EC00027F0A00EB8EC2CF05450E866EEEF2AF074
:104ED000FAEF2AF01EEC2DF0C00EB8EC2CF0140EF8
:104EE000036E000EF86E4F0EF76EC00EF66E0900E0
:104EF000F550A0EC2CF0032EFAD7899A0F0EF8EC9F
:104F000003F002EC04F0898AE8BE98EC27F0A4ECE8
:104F100027F0120E036E01EE3CF0940EB8EC2CF06C
:104F2000EE50A0EC2CF0032EFBD727EC28F012005B
:104F3000120E036E01EE3CF0000EEE6E032E9DEF9E
:104F400027F0A4EC28F01200E1EC2AF001EE3CF08E
:104F5000020E52EC29F043EC29F03A0EEE6E010EEF
:104F600052EC29F048EC29F03A0EEE6E000E52ECAD
:104F700029F048EC29F0200EEE6EEE6E060E52EC93
:104F800029F0126E1238010B3009EE6E12500F0B21
:104F90003009EE6E2F0EEE6E050E52EC29F043EC4A
:104FA00029F02F0EEE6E040E52EC29F0126E12381C
:104FB0000F0B3009EE6E12500F0B3009EE6E12001F
:104FC00054696D6520262044617465205365742002
:104FD0002020202007A81EEC2DF0DE0EB8EC2CF0CF
:104FE000200EA0EC2CF0200EA0EC2CF0020E52ECC7
:104FF00029F0126E1238030B3009A0EC2CF012507D
:105000000F0B3009A0EC2CF03A0EA0EC2CF0010EA6
:1050100052EC29F0126E1238070B3009A0EC2CF07C
:1050200012500F0B3009A0EC2CF03A0EA0EC2CF033
:10503000000E52EC29F0126E1238070B3009A0EC6A
:105040002CF012500F0B3009A0EC2CF012000E0EB9
:10505000B8EC2CF0940E206E01EE3CF0940E205C27
:10506000E926000EEA22EFCF29F02050B8EC2CF010
:10507000E7EC28F02CA895EC28F02CA09DEC28F06B
:105080002CA213D02CA631D02CA45ED02CAA000CBC
:105090002950A0EC2CF001EE3CF0940E205CE926A7
:1050A000000EEA2229C0EFFFD7D7202AA60E20182B
:1050B000940ED8B4206E960E2018D8B4202A990EDB
:1050C0002018D8B4202A9C0E2018D8B4202A9D0E6F
:1050D0002018D8B4202AA00E2018D8B4202AA30E55
:1050E0002018D8B4202A2CEF28F020062050930A4C
:1050F000A50ED8B4206EA30E2018D8B42006A00E9A
:105100002018D8B420069D0E2018D8B420069C0E76
:105110002018D8B42006990E2018D8B42006960E70
:105120002018D8B420062CEF28F0292A2950390E4F
:1051300029641200300E296E12002906300E2960F3
:105140001200390E296E120001014251070B136E35
:10515000133A43510F0B1312000E59EC29F03F5133
:10516000070B136E133A40510F0B1312010E59EC3B
:1051700029F03C51030B136E133A3D510F0B1312E0
:10518000020E59EC29F046510F0B136E133A47519A
:105190000F0B1312060E59EC29F04951010B136E37
:1051A000133A4A510F0B1312050E59EC29F04C51CA
:1051B000030B136E133A4D510F0B1312040E59ECDF
:1051C00029F0440E136E0F0E59EC29F01200FF0E59
:1051D0002C6E8150FF0B2C18D8B41200FF0A2C6ED5
:1051E00015EC2DF015EC2DF08150FF0B2C18D8A4E8
:1051F000EED700EC2DF08150FF0B2C18D8A4E7D788
:1052000081AA03D081AC20D01200800E036E15EC71
:105210002DF081BA120015EC2DF081BA120015ECB8
:105220002DF081BA1200032EF2D768EC17F0FF0EB2
:105230002C6E800E036E15EC2DF015EC2DF0032E68
:10524000FAD71EEC2DF01200800E036E15EC2DF037
:1052500081BC120015EC2DF081BC120015EC2DF074
:1052600081BC1200032EF2D783EC17F0FF0E2C6ED8
:10527000800E036E15EC2DF015EC2DF0032EFAD7F1
:105280001EEC2DF01200126E1238030B4BEF29F0BA
:10529000126E1238070B3009EE6E12500F0B3009E8
:1052A000EE6E1200899AF8EC03F002EC04F0898AA1
:1052B0001200899A8009F8EC03F01350F8EC03F01F
:1052C000898A120001018C698D69120001018F6BBE
:1052D0008E6F8D518E1BD8908E378F37000EF86EE3
:1052E000530EF76E1E0EF66E8E51F6268F51F72274
:1052F000E86AF8220900F5CF8EF10800F5508C1904
:105300008D6F8C6B8E518C1B120001018C1F8D1FB9
:105310008CC18EF18DC18CF18EC18DF11200000017
:1053200011892312329B462457AD653674BF8C48D1
:105330009DC1AF5ABED3CA6CDBE5E97EF8F7108198
:1053400001083393221A56A5472C75B7643E9CC9B1
:105350008D40BFDBAE52DAEDCB64F9FFE876210277
:10536000308B02101399672676AF443455BDAD4A91
:10537000BCC38E589FD1EB6EFAE7C87CD9F5318358
:10538000200A1291031877A7662E54B5453CBDCB71
:10539000AC429ED98F50FBEFEA66D8FDC974420437
:1053A000538D6116709F042015A9273236BBCE4C51
:1053B000DFC5ED5EFCD7886899E1AB7ABAF3528518
:1053C000430C7197601E14A1052837B3263ADECD31
:1053D000CF44FDDFEC5698E98960BBFBAA726306F7
:1053E000728F4014519D252234AB063017B9EF4E11
:1053F000FEC7CC5CDDD5A96AB8E38A789BF17387D8
:10540000620E5095411C35A3242A16B10738FFCFF0
:10541000EE46DCDDCD54B9EBA8629AF98B708408B6
:105420009581A71AB693C22CD3A5E13EF0B70840E8
:1054300019C92B523ADB4E645FED6D767CFF94897F
:105440008500B79BA612D2ADC324F1BFE03618C1C8
:1054500009483BD32A5A5EE54F6C7DF76C7EA50A5E
:10546000B48386189791E32EF2A7C03CD1B52942A8
:1054700038CB0A501BD96F667EEF4C745DFDB58B3F
:10548000A40296998710F3AFE226D0BDC13439C388
:10549000284A1AD10B587FE76E6E5CF54D7CC60C1E
:1054A000D785E51EF497802891A1A33AB2B34A4468
:1054B0005BCD695678DF0C601DE92F723EFBD68DFF
:1054C000C704F59FE41690A98120B3BBA2325AC548
:1054D0004B4C79D7685E1CE10D683FF32E7AE70EDE
:1054E000F687C41CD595A12AB0A3823893B16B4628
:1054F0007ACF485459DD2D623CEB0E701FF9F78FBF
:10550000E606D49DC514B1ABA02292B983307BC707
:105510006A4E58D5495C3DE32C6A1EF10F7815ECB4
:105520002DF015EC2DF0300EC6EC2CF015EC2DF016
:10553000300EC6EC2CF015EC2DF0300EC6EC2CF035
:10554000E9EC2CF0240EC6EC2CF015EC2DF0D0EC90
:105550002CF0280EB8EC2CF00C0EB8EC2CF0010E50
:10556000B8EC2CF0060EB8EC2CF012000C0EB8ECD7
:105570002CF0800EB8EC2CF0066A062A520EF66E5D
:105580005A0EF76E000EF86E0900F55003E0A0EC1D
:105590002CF0FAD7940EB8EC2CF00900F55003E08B
:1055A000A0EC2CF0FAD7062AD40EB8EC2CF00900A7
:1055B000F55003E0A0EC2CF0FAD707981200C00ECB
:1055C00003D0940E01D0D40EB8EC2CF0140E026E61
:1055D000200EA0EC2CF0022EFBD71200200EA0EC27
:1055E0002CF04F0EA0EC2CF06E0EA0EC2CF05AEC30
:1055F0002BF00CD0200EA0EC2CF04F0EA0EC2CF0D9
:10560000660EA0EC2CF0660EA0EC2CF051EC2BF00A
:10561000196A1200200EA0EC2CF0460EA0EC2CF023
:10562000750EA0EC2CF06C0EA0EC2CF06C0EA0EC27
:105630002CF00FD0200EA0EC2CF0480EA0EC2CF09B
:10564000610EA0EC2CF06C0EA0EC2CF0660EA0EC21
:105650002CF054EC2BF01200300EA0EC2CF06D0E60
:10566000A0EC2CF0530EA0EC2CF0650EA0EC2CF06E
:10567000630EA0EC2CF012005AEC2BF0530EA0ECB1
:105680002CF0650EA0EC2CF0630EA0EC2CF02E0E8E
:10569000A0EC2CF01200200EA0EC2CF0200EA0ECC0
:1056A0002CF0200EA0EC2CF0200EA0EC2CF0200E04
:1056B000A0EC2CF0200EA0EC2CF01200079A136E38
:1056C000300E1E6E640E135ED8A00DD01E2A640E1E
:1056D000135ED8A002D01E2A02D0640E13261E50DC
:1056E000A0EC2CF007D0640E1326200EA0EC2CF0BA
:1056F000078A00D0300E1E6E0A0E135ED8A002D0AC
:105700001E2AFAD71E5007AA06D0300AD8B402D0F3
:105710001E5001D0200EA0EC2CF00A0E13261350C0
:10572000300FA0EC2CF01200079A136E13503AE0E1
:10573000300E1E6E640E135ED8A00DD01E2A640EAD
:10574000135ED8A002D01E2A02D0640E13261E506B
:10575000A0EC2CF007D0640E1326200EA0EC2CF049
:10576000078A00D0300E1E6E0A0E135ED8A002D03B
:105770001E2AFAD71E5007AA06D0300AD8B402D083
:105780001E5001D0200EA0EC2CF00A0E1326135050
:10579000300FA0EC2CF01200200E07BA300EA0EC57
:1057A0002CF01200200EA0EC2CF0200EA0EC2CF01F
:1057B000200EA0EC2CF01200078A36C013F037C080
:1057C00014F0036A640E145E000E135AD8A002D0BF
:1057D000032AF8D7640E14261E6A0A0E035ED8A0A8
:1057E00002D01E2AFAD71E5003E0079A300903D0D0
:1057F000300907BA200EA0EC2CF00A0E0326035045
:1058000003E0079A300903D0300E07BA200EA0EC4F
:105810002CF01E6A0A0E145ED8A002D01E2AFAD7F7
:105820001E5003E0079A300904D0300907AA01D0BE
:10583000200EA0EC2CF00A0E14261450300FA0EC11
:105840002CF01200060E036ED89038323932032E37
:10585000FCD7C80EB8EC2CF0078A38C013F039C05A
:1058600014F0036A640E145E000E135AD8A002D01E
:10587000032AA8D7640E14261E6A0A0E035ED8A057
:1058800002D01E2AFAD71E5003E0079A300903D02F
:10589000300907BA200EA0EC2CF00A0E03260350A4
:1058A00003E0079A300903D0300E07BA200EA0ECAF
:1058B0002CF01E6A0A0E145ED8A002D01E2AFAD757
:1058C0001E50B3E0079A300904D0300907AA01D06E
:1058D000200EA0EC2CF00A0E14261450300FA0EC71
:1058E0002CF01200136E13380F0B1E6E0A0E1E6082
:1058F00002D0300E01D0370E1E24A0EC2CF0135035
:105900000F0B1E6E0A0E1E6002D0300E01D0370E35
:105910001E24A0EC2CF01200136E300E1E6E0A0E28
:10592000135ED8A097EF2CF01E2A8FEF2CF01E509C
:10593000A0EC2CF00A0E13243009A0EC2CF012007D
:10594000016ED0EC2CF00150F00BAEEC2CF00138D5
:10595000F00BAEEC2CF0E9EC2CF01200E83A200948
:10596000896E8B928B808B84000000008B941200D8
:10597000016ED0EC2CF00150F00BC6EC2CF001388D
:10598000F00BC6EC2CF0F9EC2CF01200E83A2009F0
:10599000896E8B908B928B84000000008B94120098
:1059A000806A0F0E926E898A8B908B828B840000A6
:1059B000000080508B94006E000000008B8400007B
:1059C000000080508B9400B6EBD78B92926A898A44
:1059D0001200A40E316E312EFED71200E9EC2CF02D
:1059E000E9EC2CF0E9EC2CF0E9EC2CF0E9EC2CF0F3
:1059F00012000A0E326EE9EC2CF0322EFCD71200A7
:105A000015EC2DF015EC2DF015EC2DF015EC2DF01E
:105A100015EC2DF015EC2DF015EC2DF015EC2DF00E
:105A200015EC2DF015EC2DF01200640E326E000016
:105A30000000E9EC2CF0322EFCD712000788010E92
:105A4000B8EC2CF0060EB8EC2CF00C0EB8EC2CF0E8
:105A500012004E6F646520446973706C6179205642
:105A600030302E31390020284329205361746F7360
:105A7000686920596173756461002020202020200E
:0E5A800020374D33544A5A2F414436475A00BE
:020000040030CA
:0100010002FC
:010003001EDE
:010005008377
:010006008178
:0200000400F00A
:020000000100FD
:00000001FF
